:020000040000FA
:06000000A1EF26F0120042
:06000800A9EF23F0120035
:06001800FCEF23F01200D2
:02082A000000CC
:04082C008150100BDC
:10083000100A01E0010E00D01200B6C0F3FFB7C0ED
:10084000F4FF00D01200B2C006F0B3C007F0B4C08D
:1008500008F0B5C009F000D0120093888186939605
:100860009288120020EC0DF08186000E00D012005C
:10087000D9CFE6FFE1CFD9FF110EE1268196AE0E6A
:10088000146E4C0E156E000E166EFE0EDBCF17F0BA
:10089000186A196A020ED890173618361936E80603
:1008A000FAE114501724F36E15501820F46E165008
:1008B0001920F86EF4CFF7FFF3CFF6FF08000A0E09
:1008C000F5CFDBFFD950FA0FE96EFF0EDA20EA6EA2
:1008D000060EEECFDBFF070EEECFDBFF080EEECFEE
:1008E000DBFF090EEECFDBFFAE0E146E4C0E156E65
:1008F000000E166EFE0EDBCF17F0186A196A020E94
:10090000D890173618361936E806FAE1145017242D
:10091000F36E15501820F46E16501920F86EF4CFAF
:10092000F7FFF3CFF6FFF62A000EF722F8220800B1
:10093000050EF5CFDBFF0A0EDB8CDBCFE6FF22ECEA
:100940000DF0E552090EDBCFE6FF22EC0DF0E5528B
:10095000080EDBCFE6FF22EC0DF0E552070EDBCFF1
:10096000E6FF22EC0DF0E552060EDBCFE6FF22ECAF
:100970000DF0E552050EDBCFE6FF22EC0DF0E5525F
:10098000FE0EDB50050802E13BEC0DF0140EF36E99
:100990000B0EF3CFDBFF0C0EDB6A3BEC0DF0DF6ED2
:1009A0000B0EDB060C0E01E2DB06FF0EDF5C08E13E
:1009B000D9500B0FE96EDACFEAFFEE50ED10EDE102
:1009C000AE0E146E4C0E156E000E166EFE0EDBCFC4
:1009D00017F0186A196A020ED890173618361936A9
:1009E000E806FAE114501724F36E15501820F46E3F
:1009F00016501920F86EF4CFF7FFF3CFF6FF020E72
:100A0000F626000EF722F8220800F550020807E14A
:100A1000010EDFCFDBFF3BEC0DF0DF6E95D0AE0EAD
:100A2000146E4C0E156E000E166EFE0EDBCF17F018
:100A3000186A196A020ED890173618361936E80661
:100A4000FAE114501724F36E15501820F46E165066
:100A50001920F86EF4CFF7FFF3CFF6FF020EF6265B
:100A6000000EF722F8220800F55001082DE10D0EC6
:100A7000DB6A0E0EDB6A0A0EF36E0F0EF3CFDBFF9E
:100A8000100EDB6A3BEC0DF0DF6ED9500D0FE96EF6
:100A9000DACFEAFFEE06000EEE5AEE5AEE5ADF50BB
:100AA00011E10D0EDBCF14F00E0EDBCF15F00F0EA3
:100AB000DBCF16F0100EDBCF17F014501510161008
:100AC0001710E0E1DF6A40D0AE0E146E4C0E156ECA
:100AD000000E166EFE0EDBCF17F0186A196A020EB2
:100AE000D890173618361936E806FAE1145017244C
:100AF000F36E15501820F46E16501920F86EF4CFCE
:100B0000F7FFF3CFF6FF020EF626000EF722F822CB
:100B10000800F550040818E13BEC0DF0E76E040EF8
:100B2000E7CFDBFF3BEC0DF0E76E030EE7CFDBFF1B
:100B30003BEC0DF0E76E020EE7CFDBFF3BEC0DF078
:100B4000E76E010EE7CFDBFFE66822EC0DF0E55221
:100B5000AE0E146E4C0E156E000E166EFE0EDBCF32
:100B600017F0186A196A020ED89017361836193617
:100B7000E806FAE114501724F36E15501820F46EAD
:100B800016501920F86EF4CFF7FFF3CFF6FF030EDF
:100B9000F626000EF722F8220800F55001E18186C2
:100BA000D9CFE9FFDACFEAFFEECF14F0EECF15F0A0
:100BB000EECF16F0EECF17F0EFCF18F0D9CFE9FF58
:100BC000DACFEAFFED50ED5018C0EDFF17C0EDFF92
:100BD00016C0EDFF15C0EDFF14C0EFFF110EE15C74
:100BE00003E200D0E16AE552E16EE552E7CFD9FFBA
:100BF0001200D9CFE6FFE1CFD9FF0E0EE126819694
:100C0000AE0E146E4C0E156E000E166EFE0EDBCF81
:100C100017F0186A196A020ED89017361836193666
:100C2000E806FAE114501724F36E15501820F46EFC
:100C300016501920F86EF4CFF7FFF3CFF6FF080037
:100C40000B0EF5CFDBFFD950FA0FE96EFF0EDA205D
:100C5000EA6E070EEECFDBFF080EEECFDBFF090ECC
:100C6000EECFDBFF0A0EEECFDBFFAE0E146E4C0EA6
:100C7000156E000E166EFE0EDBCF17F0186A196A9D
:100C8000020ED890173618361936E806FAE11450D5
:100C90001724F36E15501820F46E16501920F86EB4
:100CA000F4CFF7FFF3CFF6FFF62A000EF722F82273
:100CB0000800060EF5CFDBFF0B0EDB8CDBCFE6FF6B
:100CC0005FEC0DF0E5520A0EDBCFE6FF5FEC0DF0B6
:100CD000E552090EDBCFE6FF5FEC0DF0E552080EA2
:100CE000DBCFE6FF5FEC0DF0E552070EDBCFE6FF52
:100CF0005FEC0DF0E552060EDBCFE6FF5FEC0DF08A
:100D0000E552FE0EDB50050802E1A1EC0DF0140ED9
:100D1000F36E0C0EF3CFDBFF0D0EDB6AA1EC0DF0D2
:100D2000E76E010EE7CFDBFF0C0EDB060D0E01E2D6
:100D3000DB06010EDB50FF0808E1D9500C0FE96E0D
:100D4000DACFEAFFEE50ED10E9E1AE0E146E4C0E74
:100D5000156E000E166EFE0EDBCF17F0186A196ABC
:100D6000020ED890173618361936E806FAE11450F4
:100D70001724F36E15501820F46E16501920F86ED3
:100D8000F4CFF7FFF3CFF6FF020EF626000EF722A0
:100D9000F8220800F55002080DE1010EDB50E76E65
:100DA000020EE7CFDBFFA1EC0DF0E76E010EE7CFFF
:100DB000DBFF85D0AE0E146E4C0E156E000E166E57
:100DC000FE0EDBCF17F0186A196A020ED89017369C
:100DD00018361936E806FAE114501724F36E155048
:100DE0001820F46E16501920F86EF4CFF7FFF3CFE9
:100DF000F6FF020EF626000EF722F8220800F55044
:100E000001081DE10C0EDB680D0EDB68A1EC0DF096
:100E1000E76E010EE7CFDBFF0C0EDB060D0E01E2E5
:100E2000DB06010EDB5008E1D9500C0FE96EDACF7A
:100E3000EAFFEE50ED10EAE1010EDB6A40D0AE0EA3
:100E4000146E4C0E156E000E166EFE0EDBCF17F0F4
:100E5000186A196A020ED890173618361936E8063D
:100E6000FAE114501724F36E15501820F46E165042
:100E70001920F86EF4CFF7FFF3CFF6FF020EF62637
:100E8000000EF722F8220800F550040818E1A1EC42
:100E90000DF0E76E050EE7CFDBFFA1EC0DF0E76E7E
:100EA000040EE7CFDBFFA1EC0DF0E76E030EE7CFFA
:100EB000DBFFA1EC0DF0E76E020EE7CFDBFFE6688B
:100EC0005FEC0DF0E552AE0E146E4C0E156E000E7A
:100ED000166EFE0EDBCF17F0186A196A020ED89054
:100EE000173618361936E806FAE114501724F36E4F
:100EF00015501820F46E16501920F86EF4CFF7FF35
:100F0000F3CFF6FF030EF626000EF722F8220800B4
:100F1000F55001E18186010EDBCF14F0020EDBCF2C
:100F200015F0030EDBCF16F0040EDBCF17F0050E25
:100F3000DBCF18F0D9CFE9FFDACFEAFFED50ED5063
:100F400018C0EDFF17C0EDFF16C0EDFF15C0EDFF97
:100F500014C0EFFF0E0EE15C03E200D0E16AE5523F
:100F6000E16EE552E7CFD9FF1200D9CFE6FFE1CF1E
:100F7000D9FF0E0EE126DE6A020EDD6EDB6AF36E2D
:100F8000030EF3CFDBFF040EDB6A050EDB6AF90EFE
:100F9000DBCF08F0FA0EDBCF09F0060E08C0DBFF4E
:100FA000070E09C0DBFFD950FB0FE96EFF0EDA20F8
:100FB000EA6E080EEECFDBFF090EEECFDBFF0A0E66
:100FC000EECFDBFF0B0EEECFDBFF010EF36E0C0E50
:100FD000F3CFDBFFD9CFE6FFDACFE6FF20D8E5522B
:100FE000E552E76E0D0EE7CFDBFFDB5003E1010EAC
:100FF0000AD006D00D0EDB50FF0802E1000E03D030
:10100000E9D7000E00D0146E0E0EE15C02E2E16A38
:10101000E552E16E1450E552E7CFD9FF1200D9CF67
:10102000E6FFE1CFD9FF060EE126FD0EDBCFE9FF9B
:10103000FE0EDBCFEAFF0C0EE926000EEA22EF508F
:10104000FF0A01E1A3D1010A01E170D1FC0A01E12B
:10105000FED0010A01E1BBD0020A05E0010A01E06D
:1010600095D1000E9BD10001CB6B020ECC6FFD0E13
:10107000DBCFE9FFFE0EDBCFEAFFEECFBEF0EECF17
:10108000BFF0EECFC0F0EECFC1F0EECFC2F0EECFAA
:10109000C3F0EECFC4F0EECFC5F0EECFC6F0EECF8A
:1010A000C7F0EECFC8F0EECFC9F0EFCFCAF0B8511D
:1010B00008E1090ED890C637C737C837C937E806E0
:1010C000F9E1D880000E0001C055020EC155000E96
:1010D000C255000EC3552CE3010ED16FC6C0E6FF0A
:1010E000C7C0E6FFC8C0E6FFC9C0E6FF080EE66E4F
:1010F00038EC04F0EECF14F0EECF15F0EECF16F092
:10110000EECF17F0EECF18F0196E050EE15E195014
:10111000010E14C0DBFF020E15C0DBFF030E16C06C
:10112000DBFF040E17C0DBFF050E18C0DBFF2AD063
:10113000D16BC6C0E6FFC7C0E6FFC8C0E6FFC9C0A6
:10114000E6FF090EE66E38EC04F0EECF14F0EECFB9
:1011500015F0EECF16F0EECF17F0EECF18F0196EB7
:10116000050EE15E1950010E14C0DBFF020E15C022
:10117000DBFF030E16C0DBFF040E17C0DBFF050EFE
:1011800018C0DBFF010EDB500EE0FD0EDBCFE9FFE8
:10119000FE0EDBCFEAFF0C0EE926000EEA22FE0E61
:1011A000EF6E010EFBD00001CD6BCE6B040ECF6F46
:1011B000D06BFD0EDBCFE9FFFE0EDBCFEAFF0C0E9E
:1011C000E926000EEA22030EEF6E010EE7D00001C1
:1011D000CD51CE11CF11D0112CE0CD07000ECE5B3A
:1011E000CF5BD05B3BEC0DF0DF6EFF0EDF5C1FE0F2
:1011F000FE0EDF5C0EE1FD0EDBCFE9FFFE0EDBCF66
:10120000EAFF0C0EE926000EEA22020EEF6EC6D0AF
:101210001ED0FD0EDBCFE9FFFE0EDBCFEAFF0C0E8A
:10122000E926000EEA22FE0EEF6E010EB7D0010E87
:10123000B5D0FD0EDBCFE9FFFE0EDBCFEAFF0C0ED3
:10124000E926000EEA22FE0EEF6E010EA7D0000185
:10125000C051C111C211C3114BE0FD0EDBCFE9FF3C
:10126000FE0EDBCFEAFFEECFBEF0EDCFBFF0FD0EFE
:10127000DBCFE9FFFE0EDBCFEAFF060EE926000E0C
:10128000EA22EECFC4F0EDCFC5F0BEC014F0BFC06F
:1012900015F0166A176A1450C05F1550C15B1650DE
:1012A000C25B1750C35BBE51CB5FBF51CC5B82D8D2
:1012B0000001CB51CC1119E1DEDBDDDB0001C051B7
:1012C000C111C211C3110CE0FD0EDBCFE9FFFE0E10
:1012D000DBCFEAFF0C0EE926000EEA22030EEF6ECA
:1012E000CB6B020ECC6F010E59D0020E57D01ED020
:1012F000D1510CE1E66AE66AE66AE66A050EE66E38
:1013000038EC04F0146E050EE15E14508186E66838
:1013100099DBE552FD0EDBCFE9FFFE0EDBCFEAFFE6
:101320000C0EE926000EEA22EF6A38D0FD0EDBCF64
:10133000E9FFFE0EDBCFEAFF0C0EE926000EEA22E3
:10134000EF68E66AE66AE66AE66A050EE66E38EC7B
:1013500004F0EECF14F0EECF15F0EECF16F0EECF96
:1013600017F0EECF18F0196E050EE15E1950010E60
:1013700014C0DBFF020E15C0DBFF030E16C0DBFF3F
:10138000040E17C0DBFF050E18C0DBFF8186E66880
:1013900059DBE552FF0E02D0FF0E00D0146E060E90
:1013A000E15C02E2E16AE552E16E1450E552E7CFFA
:1013B000D9FF12000001BE51BF1101E12ED0E9CFCB
:1013C000D2F0EACFD3F0F3CFD4F0F4CFD5F0BEC053
:1013D000F3FFBFC0F4FFC4C0E9FFC5C0EAFFC950B6
:1013E000E86E9E96C96806D09EA6FED79E96C95006
:1013F000C968EE6E000EF306F45AF350F410F4E1EF
:101400009EA6FED7C9CFEEFF9E96D4C0F3FFD5C0EF
:10141000F4FFD2C0E9FFD3C0EAFF1200D9CFE6FF44
:10142000E1CFD9FF090EE126FD0EDBCFE9FFFE0E6D
:10143000DBCFEAFF0C0EE926000EEA22EF50FE0A8F
:1014400001E100D2FA0A01E1DBD1070A01E174D11E
:10145000010A01E1FED0030A05E0010A01E00DD214
:10146000000E1BD20001D76B020ED86FFD0EDBCF32
:10147000E9FFFE0EDBCFEAFFEECFBEF0EECFBFF00E
:10148000EECFC0F0EECFC1F0EECFC2F0EECFC3F0A2
:10149000EECFC4F0EECFC5F0EECFC6F0EECFC7F082
:1014A000EECFC8F0EECFC9F0EFCFCAF0D880000E73
:1014B000C055020EC155000EC255000EC35503E3C0
:1014C0000A0EDD6F73D00B0EDD6FC0C014F0C1C00B
:1014D00015F0C2C016F0C3C017F0090ED89017322D
:1014E000163215321432E806F9E114C0DFFF010E9E
:1014F00015C0DBFF020E16C0DBFF030E17C0DBFFBB
:10150000D9CFE9FFDACFEAFFEECF14F0EECF15F036
:10151000EECF16F0EFCF17F014501510161017106D
:1015200009E1D9CFE9FFDACFEAFFEE2A000EEE2279
:10153000EE22EE22E66AE66AE66AE66A0F0EE66EDA
:1015400038EC04F0EECF14F0EECF15F0EECF16F03D
:10155000EECF17F0EECF18F0196E050EE15E1950C0
:10156000040E14C0DBFF050E15C0DBFF060E16C00F
:10157000DBFF070E17C0DBFF080E18C0DBFF040EF1
:10158000DB5014E1D9CFE9FFDACFEAFFEECFE6FF77
:10159000EECFE6FFEECFE6FFEFCFE6FF130EE66EEF
:1015A00038EC04F0146E050EE15E14500001B851E1
:1015B00008E1090ED890C637C737C837C937E806DB
:1015C000F9E1C6C0E6FFC7C0E6FFC8C0E6FFC9C074
:1015D000E6FFDDC0E6FF38EC04F0EECF14F0EECF0E
:1015E00015F0EECF16F0EECF17F0EECF18F0196E23
:1015F000050EE15E1950040E14C0DBFF050E15C088
:10160000DBFF060E16C0DBFF070E17C0DBFF080E60
:1016100018C0DBFF040EDB500EE0FD0EDBCFE9FF50
:10162000FE0EDBCFEAFF0C0EE926000EEA22EF6881
:10163000FF0E33D10CD0FD0EDBCFE9FFFE0EDBCF6A
:10164000EAFF0C0EE926000EEA22020EEF6E020EF1
:1016500024D10001D75102E1020ED8190CE10B0E82
:10166000DD5D05E1FC0EE66EEDD9E55204D0FE0E1F
:10167000E66EE8D9E552FD0EDBCFE9FFFE0EDBCFCB
:10168000EAFFEECFBEF0EDCFBFF0FD0EDBCFE9FFFE
:10169000FE0EDBCFEAFF060EE926000EEA22EECFB1
:1016A000C4F0EDCFC5F0BEC014F0BFC015F0166A8F
:1016B000176A14500001C05F1550C15B1650C25B21
:1016C0001750C35BBE51D75FBF51D85BF2D8000142
:1016D000D751D8112FE1D76B020ED86FE668B2D977
:1016E000E552E668AFD9E552C6D91F0B05080EE0F2
:1016F000FD0EDBCFE9FFFE0EDBCFEAFF0C0EE92685
:10170000000EEA22FE0EEF6E030EC7D0FD0EDBCFF9
:10171000E9FFFE0EDBCFEAFF0C0EE926000EEA22FF
:10172000030EEF6E0001D96BDA6B0A0EDB6FDC6B18
:10173000030EB3D0020EB1D00001D951DA11DB1182
:10174000DC1150E0D907000EDA5BDB5BDC5BE6689E
:1017500079D9E55290D90001D66FD65141E0C051F8
:10176000C111C211C3112EE1D96BDA6B0A0EDB6F06
:10177000DC6B0B0EDD5D16E1FD0EE66E63D9E55206
:10178000E66860D9E552FD0EDBCFE9FFFE0EDBCF48
:10179000EAFF0C0EE926000EEA22040EEF6E030E9D
:1017A0007CD010D08186E6684DD9E552FD0EDBCFA6
:1017B000E9FFFE0EDBCFEAFF0C0EE926000EEA225F
:1017C000EF6A6BD0FD0EDBCFE9FFFE0EDBCFEAFF49
:1017D0000C0EE926000EEA22020EEF6E5ED010D04B
:1017E000030E5BD0FD0EDBCFE9FFFE0EDBCFEAFF81
:1017F0000C0EE926000EEA22FE0EEF6E030E4DD00F
:101800000001D951DA11DB11DC111CE0D907000EFF
:10181000DA5BDB5BDC5B2FD90001D66FD65110E0C1
:101820008186E6680FD9E552FD0EDBCFE9FFFE0E9B
:10183000DBCFEAFF0C0EE926000EEA22EF6A2DD07C
:10184000030E2BD0E66AE66AE66AE66A050EE66EE5
:1018500038EC04F0146E050EE15E14508186E668E3
:10186000F1D8E552FD0EDBCFE9FFFE0EDBCFEAFF3C
:101870000C0EE926000EEA22EF68FF0E0ED0FD0ED8
:10188000DBCFE9FFFE0EDBCFEAFF0C0EE926000EF0
:10189000EA22FE0EEF6E030E00D0146E090EE15C1C
:1018A00002E2E16AE552E16E1450E552E7CFD9FF5A
:1018B00012000001BE51BF1101E12AD0E9CFDFF0D3
:1018C000EACFE0F0F3CFE1F0F4CFE2F0BEC0F3FFF7
:1018D000BFC0F4FFC4C0E9FFC5C0EAFFEE5003D0AB
:1018E000EE509EA6FED79E96C96E000EF306F45AE1
:1018F000F350F410F5E19EA6FED7C9CFDEF09E9618
:10190000E1C0F3FFE2C0F4FFDFC0E9FFE0C0EAFF9F
:101910001200D9CFE6FFE1CFD9FFE652F80EDB5037
:1019200013E1FB0EDBCF14F0FC0EDBCF15F0FD0E48
:10193000DBCF16F0FE0EDBCF17F01450151016108B
:10194000171002E1000E31D00001E36B020EE46FCC
:10195000E56BE66FE76BE86BF90EDBCFE9F0FA0EAB
:10196000DBCFEAF0FB0EDBCFEBF0FC0EDBCFECF0D5
:10197000FD0EDBCFEDF0FE0EDBCFEEF0010EEF6FD4
:10198000E30EE66E000EE66E49DDE552E552DF6ECF
:10199000DF5003E1010E09D005D0FF0EDF5C02E14C
:1019A000000E03D0EDD7010E00D0E552E552E7CF8F
:1019B000D9FF12008050100B01E0010E00D0120080
:1019C000D9CFE6FFE1CFD9FF050EE126FE0EDB50B1
:1019D000DF6EDF50DF06000927E06B0EF36E010EAD
:1019E000F3CFDBFF170EF36E020EF3CFDBFF030E18
:1019F000DB6A040EDB6AD950010FE96EDACFEAFF29
:101A0000EFCF14F0EE06000EEFCF15F0EE5AEFCF49
:101A100016F0EE5AEFCF17F0EF5A145015101610BB
:101A2000171001E0E8D7D5D7000000D0050EE15C23
:101A300002E2E16AE552E16EE552E7CFD9FF12001A
:101A4000C69A1200D9CFE6FFE1CFD9FFE652C950BE
:101A5000DF6E9E96FE0EDB50C96EC6AE03D0FF0E43
:101A600005D002D09EA6FED7000E00D0E552E5526A
:101A7000E7CFD9FF1200D9CFE6FFE1CFD9FFE65279
:101A8000C950DF6E9E96C9689EA6FED7C95000D089
:101A9000E552E552E7CFD9FF1200D9CFE6FFE1CFFB
:101AA000D9FFC76AC66AFE0EDB50C612C78C939276
:101AB000949E9380C68AE552E7CFD9FF1200D9CF12
:101AC000E6FFE1CFD9FF020EE1268A928B8E939238
:101AD000949EDF6A080EDF5C25E28A92FE0EDBAE82
:101AE00002D08B8E01D08B9EDB50020DFE0EF3CF09
:101AF000DBFFDE52010EDD6E010EDBCFF3FFDB06F6
:101B0000F350000901E0F8D78A82DE52010EDD6E43
:101B1000010EDBCFF3FFDB06F350000901E0F8D73D
:101B2000DF2AD8D78A92000E146E020EE15C03E21F
:101B300000D0E16AE552E16E1450E552E7CFD9FFDB
:101B40001200D9CFE6FFE1CFD9FF030EE126020E46
:101B5000DB6A8B8E949E93808A929392DF6A080E42
:101B6000DF5C22E28A92DE52010EDD6E010EDBCFD7
:101B7000F3FFDB06F350000901E0F8D78A82DE525A
:101B8000010EDD6E010EDBCFF3FFDB06F350000923
:101B900001E0F8D7020EDB50020D020EF3CFDBFF9F
:101BA00081B0DB2ADF2ADBD78A92020EDB50146E6B
:101BB000030EE15C03E200D0E16AE552E16E1450ED
:101BC000E552E7CFD9FF1200C66A8A928B8E9392B4
:101BD000949E1200D9CFE6FFE1CFD9FF230EE12674
:101BE0000001B96BBA6BB26BB36BB46BB56BB86B0E
:101BF0008186EADF1E0EE66EE3DEE5528186DE6A4E
:101C0000DD6ADECF14F0DDCF15F00A0E145C000E95
:101C1000155808E2E66853DFE552DF2A010E01E3BA
:101C2000DB2AEFD7640EDE6EDD6A8186E66847DF69
:101C3000E5528196DF06010E01E2DB06E66AE66AFE
:101C4000E66AE66AE66AF9EC05F0EECF14F0EECF4C
:101C500015F0EECF16F0EECF17F0EECF18F0196EAC
:101C6000050EE15E1950020E14C0DBFF030E15C015
:101C7000DBFF040E16C0DBFF050E17C0DBFF060EF0
:101C800018C0DBFF020EDB0407E0D9CFE9FFDACF93
:101C9000EAFFEE50ED10C9E1D9CFE9FFDACFEAFF54
:101CA000EE50ED105FE18186E66809DFE55281962E
:101CB000E66AE66AE66AE66A050EE66EF9EC05F0A3
:101CC000EECF14F0EECF15F0EECF16F0EECF17F00A
:101CD000EECF18F0196E050EE15E1950020E14C019
:101CE000DBFF030E15C0DBFF040E16C0DBFF050E85
:101CF00017C0DBFF060E18C0DBFFE66AE66AE66A7D
:101D0000E66AE66AF9EC05F0EECF14F0EECF15F0D6
:101D1000EECF16F0EECF17F0EECF18F0196E050EDD
:101D2000E15E1950020E14C0DBFF030E15C0DBFF8D
:101D3000040E16C0DBFF050E17C0DBFF060E18C031
:101D4000DBFF020EDB040DE00001020EB96FB90EDD
:101D5000146E000E156E14C0F3FF15C0F4FF4BD3C4
:101D600000D000D0AA0EE66E010EE66EE66AE66AC4
:101D7000020EE66EF9EC05F0EECF14F0EECF15F0A2
:101D8000EECF16F0EECF17F0EECF18F0196E050E6D
:101D9000E15E1950020E14C0DBFF030E15C0DBFF1D
:101DA000040E16C0DBFF050E17C0DBFF060E18C0C1
:101DB000DBFF14680F0E156E166A176AD950030FF1
:101DC000E96EDACFEAFFEE501416EE501516EE501B
:101DD0001616EE501716AA0E141806E1010E151865
:101DE00003E1165001E1175001E0C3D0D950020FB2
:101DF000E96EDACFEAFFEF50040B01E0BAD0E66AF1
:101E0000E66AE66AE66A100EE66EF9EC05F0EECFD9
:101E100014F0EECF15F0EECF16F0EECF17F0EECFB8
:101E200018F0196E050EE15E1950020E14C0DBFFAA
:101E3000030E15C0DBFF040E16C0DBFF050E17C036
:101E4000DBFF060E18C0DBFFDE6ADD6ADECF14F0B2
:101E5000DDCF15F0FF0E145CFF0E15583BE2E66A6D
:101E6000E66AE66AE66A0F0EE66EF9EC05F0146EB5
:101E7000050EE15E1450E66AE66AE66A400EE66E1A
:101E8000120EE66EF9EC05F0EECF14F0EECF15F081
:101E9000EECF16F0EECF17F0EECF18F0196E050E5C
:101EA000E15E1950020E14C0DBFF030E15C0DBFF0C
:101EB000040E16C0DBFF050E17C0DBFF060E18C0B0
:101EC000DBFF020EDB5001E105D0DF2A010E01E34A
:101ED000DB2ABCD7DECF14F0DDCF15F0FF0E145C8B
:101EE000FF0E155803E30001020EB96FE66AE66AB9
:101EF000E66AE66A100EE66EF9EC05F0EECF14F035
:101F0000EECF15F0EECF16F0EECF17F0EECF18F0C3
:101F1000196E050EE15E1950020E14C0DBFF030EB0
:101F200015C0DBFF040E16C0DBFF050E17C0DBFF7C
:101F3000060E18C0DBFF146A156A166A400E176E8B
:101F4000D950030FE96EDACFEAFFEE501416EE50C7
:101F50001516EE501616EE501716145015101610D2
:101F6000171004E00001010EB86F02D00001B86B39
:101F70004AD08186010EE66E23DDE552819600018E
:101F8000B86BDE681F0EDD6EE66AE66AE66AE66A30
:101F9000010EE66EF9EC05F0EECF14F0EECF15F081
:101FA000EECF16F0EECF17F0EECF18F0196E050E4B
:101FB000E15E1950020E14C0DBFF030E15C0DBFFFB
:101FC000040E16C0DBFF050E17C0DBFF060E18C09F
:101FD000DBFFDF06010E01E2DB06020EDB5007E04D
:101FE000D9CFE9FFDACFEAFFEE50ED10CDE1D9CF3E
:101FF000E9FFDACFEAFFEE50ED1005E10001020E35
:10200000B96F818600D08186E66A47DDE552819608
:10201000140EDE6EDD6AE66AE66AE66AE66A030EBA
:10202000E66E38EC04F0EECF14F0EECF15F0EECF04
:1020300016F0EECF17F0EECF18F0196E050EE15E38
:102040001950020E14C0DBFF030E15C0DBFF040E97
:1020500016C0DBFF050E17C0DBFF060E18C0DBFF46
:10206000DF06010E01E2DB06020EDB5007E0D9CFEE
:10207000E9FFDACFEAFFEE50ED10CDE1D9CFE9FF6D
:10208000DACFEAFFEE50ED1001E00DD00001020EB4
:10209000B96F8186B90E146E000E156E14C0F3FF71
:1020A00015C0F4FFA8D11C0EDB6A1B0EDB6A140EF0
:1020B000F36E1B0EDBCFF4FFF350F45C20E2DBDCAD
:1020C000E66ED950070F146EDACF15F01C0EDB50F8
:1020D0000F011424E96E000E1520EA6EE552E75058
:1020E000EF6E1C0EDB2A1B0EDB5006E1070EDB50E9
:1020F000FE0802E11C0EDB6A1B0EDB2AD8D70001AA
:10210000B66B020EB76FBB6BBC6FBA81070EDB50AC
:10211000C00B60E00E0EDBCF14F0156A166A176A6A
:102120003F0E1416156A166A176A100E1F0B07E089
:10213000D8901436153616361736E806F9E10F0E24
:10214000DBCF18F018C019F0186A1A6A1B6A185009
:102150001412195015121A5016121B501712100E85
:10216000DBCF1CF01D6A1E6A1F6A1C5014121D5022
:1021700015121E5016121F5017121D0E14C0DBFF31
:102180001E0E15C0DBFF1F0E16C0DBFF200E17C092
:10219000DBFF1D0EDBCFB2F01E0EDBCFB3F01F0E48
:1021A000DBCFB4F0200EDBCFB5F00001B22B000E78
:1021B000B323B423B5230A0ED890B237B337B4375C
:1021C000B537E806F9E10001B207000EB35BB45B76
:1021D000B55BE5D00D0EDBCF14F0156A166A176AF1
:1021E000100E1F0B07E0D89014361536163617362A
:1021F000E806F9E10E0EDBCF18F018C019F0186AE6
:102200001A6A1B6A18501412195015121A50161215
:102210001B5017120F0EDBCF1CF01D6A1E6A1F6ABF
:102220001C5014121D5015121E5016121F5017125A
:102230001D0E14C0DBFF1E0E15C0DBFF1F0E16C0E7
:10224000DBFF200E17C0DBFFD9501D0FE96EDACF80
:10225000EAFFC00EEE16EE52030EEE16EE6A1D0EEB
:10226000DBCF14F01E0EDBCF15F01F0EDBCF16F008
:10227000200EDBCF17F0060ED8901732163215322B
:102280001432E806F9E11D0E14C0DBFF1E0E15C066
:10229000DBFF1F0E16C0DBFF200E17C0DBFF100E8A
:1022A000DB50030BE824146E110EDB50800BE84466
:1022B000010B1410E76E210EE7CFDBFF0C0EDB5095
:1022C0000F0BE76E220EE7CFDBFFDB50F70F146E2C
:1022D000010E145204E0E846FE0B1406FCE1E76E22
:1022E000220EE7CFDBFFDBCF20F0216A226A236AD0
:1022F000210EDB50020FAFEC26F0F3CF1CF0F4CF31
:102300001DF01E6A1F6A010E186E196A1A6A1B6A8E
:10231000D9501D0FE96EDACFEAFFEE501826EE50C5
:102320001922EE501A22EE501B2218C006F019C0D6
:1023300007F01AC008F01BC009F01CC00BF01DC04C
:102340000CF01EC00DF01FC00EF01FEC26F002C0F6
:1023500014F003C015F004C016F005C017F014C047
:1023600006F015C007F016C008F017C009F020C02D
:102370000BF021C00CF022C00DF023C00EF01FECBA
:1023800026F002C0B2F003C0B3F004C0B4F005C040
:10239000B5F00001B207000EB35BB45BB55BE66A53
:1023A000E66AE66AE66A110EE66E38EC04F0146E30
:1023B000050EE15E1450B6C014F0B7C015F0166AF1
:1023C000176A14C0E6FF15C0E6FF16C0E6FF17C087
:1023D000E6FF070EE66E38EC04F0186E050EE15EBF
:1023E00018508186B90E146E000E156E14C0F3FFDE
:1023F00015C0F4FF00D0230EE15C02E2E16AE55271
:0A240000E16EE552E7CFD9FF1200AC
:06240A00D9CFE6FFE1CF8F
:10241000D9FFE652A09A6A6A686A706A010EE66E8F
:10242000E66AE66A710EE66E0F0EE66E05EC26F0C1
:10243000146E050EE15E1450160E6F6E9F0E6B6EDD
:102440007B0E696EDF6ADF50146E156A080E145C2D
:10245000000E155810E2DF50040DF3CFE9FFF4CF62
:10246000EAFF000EE926040EEA22EE6AEE6AEE6A40
:10247000EE6ADF2AE8D76D8C6E6A6D986D9C68A64F
:1024800007D068960101146B196B1A6B1B6BF7D799
:102490000101010E2C6F2D6F2E6B2F6B226BDF6AEB
:1024A000020EDF5C26E2EA6ADF34FE0BEA36E96EF2
:1024B0000B0EE926010EEA22EE6AED6AEA6ADF34C3
:1024C000FE0BEA36E96E070EE926010EEA22EE6AF5
:1024D000ED6ADF50EA6A260FE96E010EEA22EF6A22
:1024E000DF50EA6A280FE96E010EEA22EF6ADF2A5E
:1024F000D7D70101080E0B6F040E0C6F160E706E0D
:102500000401200E026F040E036F080E016F840E8B
:10251000006F0101016B006BE552E552E7CFD9FF77
:102520001200D9CFE6FFE1CFD9FFE6520101000545
:1025300007E16DBA05D0686A69806988020E006F8C
:102540006850040B06E06950040B03E06894FAEC51
:1025500018F06DA202D0A19A97D06850010B09E043
:102560006950010B06E051DFA08A0101040E006FE3
:1025700068906850100B06E06950100B03E0E5EC22
:1025800018F0689868AC19D069AC0FD0010EE66EEF
:10259000E66A000EE66EE66A730EE66EE66A62ECC6
:1025A00024F0146E060EE15E1450689C01012A515D
:1025B00001E02A072A5101E10BDA6850200B05E0FF
:1025C0006950200B02E0CCEC18F06850020B13E0CD
:1025D0006950020B10E0010EE66EE66A000EE66E30
:1025E000E66AE6687F0EE66E62EC24F0146E060E74
:1025F000E15E14506A6A040E0101E76E0019E8AE4C
:1026000002D0E73402D0E750005D02E2A19A3CD04C
:1026100069A639D0DF6A040EDF5C35E268A632D0E5
:102620006CCF23F101012351780BE842E842E842E4
:10263000246F689623B508D02451EA6A280FE96E02
:10264000010EEA22EF7007D02451EA6A260FE96EE4
:10265000010EEA22EF70245103E111EC19F010D0C1
:10266000000EE66EE66A230EE66E010EE66E720E50
:10267000E66EE66A62EC24F0146E060EE15E14501B
:10268000DF2AC9D700D0A19AE552E552E7CFD9FF9A
:102690001200D9CFE6FFE1CFD9FF020EE126FD0EF1
:1026A000DBA407D0E66AFE0EDBCFE6FF22DAE552B6
:1026B000E552FD0EDBA208D0010EE66EFE0EDBCF6A
:1026C000E6FF17DAE552E552FE0EDB50156A700F91
:1026D000146E0F0E152214C0DEFF15C0DDFFDECF15
:1026E000E9FFDDCFEAFFFD0EDBCFEFFF020EE15C7D
:1026F00002E2E16AE552E16EE552E7CFD9FF12004E
:10270000D9CFE6FFE1CFD9FF020EE126FD0EDB5067
:102710000FE0FE0EEA6ADB34FE0BEA36E96E0B0EC2
:10272000E926010EEA22EECFDEFFEDCFDDFF0ED06F
:10273000FE0EEA6ADB34FE0BEA36E96E070EE92686
:10274000010EEA22EECFDEFFEDCFDDFFD9CFE9FFAC
:10275000DACFEAFFEE50ED1003E1F36AF46A49D0F4
:10276000DECFE9FFDDCFEAFF020EE926000EEA2206
:10277000FB0EDBCFEEFFFC0EDBCFEDFFDECFE9FF84
:10278000DDCFEAFFEE52FA0EDBCFEFFF400E146E04
:10279000DECFE9FFDDCFEAFF1450EF16880E146E8E
:1027A000DECFE9FFDDCFEAFF1450EF12FD0EDB5064
:1027B0000CE0FE0EEA6ADB34FE0BEA36E96E0B0E25
:1027C000E926010EEA22EF740BD0FE0EEA6ADB3432
:1027D000FE0BEA36E96E070EE926010EEA22EF74D7
:1027E000DECF14F0DDCF15F014C0F3FF15C0F4FFF9
:1027F00000D0020EE15C02E2E16AE552E16EE552D0
:10280000E7CFD9FF1200D9CFE6FFE1CFD9FF020E03
:10281000E126FE0EDB5020E105C1E9FF06C1EAFF1B
:10282000EE52080EEF6E05C1E9FF06C1EAFF020E87
:10283000E926000EEA22200EEE6E040EED6E05C1B2
:10284000E9FF06C1EAFF8C0EEF6E0BC1E9FF0CC178
:10285000EAFF840EEF6E3DD0FD0EDB50E824166ECD
:10286000FE0EDB50040DF3501624040DF3CF14F0CC
:10287000F4CF15F0000E1426040E152214C0DEFF4E
:1028800015C0DDFF840E146EDECFE9FFDDCFEAFF59
:102890001450EF12FD0EDB50E824166EFE0EDB50D6
:1028A000040DF3501624010F040DF3CF14F0F4CFF0
:1028B00015F0000E1426040E152214C0DEFF15C0FC
:1028C000DDFF840E146EDECFE9FFDDCFEAFF14508A
:1028D000EF12020EE15C02E2E16AE552E16EE552BE
:1028E000E7CFD9FF1200D9CFE6FFE1CFD9FF6DA81E
:1028F0004ED0FE0EEA6ADB34FE0BEA36E96E0B0EB2
:10290000E926010EEA22EE50EFCFEAFFE96E400E13
:10291000EE16EE6AEE6AEE6AFE0EEA6ADB34FE0B33
:10292000EA36E96E0B0EE926010EEA22EE50EFCFF1
:10293000EAFFE96EEE7CFE0EEA6ADB34FE0BEA3655
:10294000E96E0B0EE926010EEA22EF74400E146EBA
:10295000FE0EEA6ADB34FE0BEA36E96E0B0EE92660
:10296000010EEA22EE50EFCFEAFFE96E1450EF16A7
:10297000FE0EEA6ADB34FE0BEA36E96E0B0EE92640
:10298000010EEA22EE50EFCFEAFFE96EEF7CE5524E
:10299000E7CFD9FF12006D6A696A0101006B00D0B0
:1029A00012000101005113E16D6A696A160E6F6E23
:1029B0009F0E6B6E7B0E696ED08EA28AA08AF28EFD
:1029C0006DB602D06D86FCD70101010E006F1200BA
:1029D00001012C514DE1010E2C6F2D5149E1010EE9
:1029E0002D6F020E105D0DE10BC1E9FF0CC1EAFF76
:1029F000EE52EF6A0BC1E9FF0CC1EAFFC80EEF6EA1
:102A000037D0100535E1256B03C1E9FF04C1EAFFAA
:102A1000EE52080EEF6E03C1E9FF04C1EAFF020E99
:102A2000E926000EEA22200EEE6E040EED6E03C1C2
:102A3000E9FF04C1EAFF840EEF6E010E256F05C1A8
:102A4000E9FF06C1EAFFEE52080EEF6E05C1E9FF8D
:102A500006C1EAFF020EE926000EEA22200EEE6E03
:102A6000040EED6E05C1E9FF06C1EAFF800EEF6EB0
:102A7000120001012E6B2F6B020E105D1AE105C1D1
:102A8000E9FF06C1EAFFEE52080EEF6E05C1E9FF4D
:102A900006C1EAFF020EE926000EEA22280EEE6EBB
:102AA000040EED6E05C1E9FF06C1EAFFC80EEF6E28
:102AB0001FD015510401265D01011651040127594B
:102AC00004E226C415F127C416F1D1D80BC1E9FFE1
:102AD0000CC1EAFF020EE926000EEA22280EEE6E75
:102AE000040EED6E0BC1E9FF0CC1EAFFC80EEF6EDC
:102AF0001200D9CFE6FFE1CFD9FF020EE126000E8A
:102B0000DE6E040EDD6EFD0EDB50E824166EFE0E4A
:102B1000DB50040DF3501624040DF3CF14F0F4CF62
:102B200015F0D9CFE9FFDACFEAFF1450EE261550A1
:102B3000ED22DECFE9FFDDCFEAFFEF9EFD0EDB5099
:102B40000FE1FE0EEA6ADB34FE0BEA36E96E070E91
:102B5000E926010EEA22DECFEEFFDDCFEDFF0ED03B
:102B6000FE0EEA6ADB34FE0BEA36E96E0B0EE9264E
:102B7000010EEA22DECFEEFFDDCFEDFFDECFE9FF73
:102B8000DDCFEAFFEF9CDECFE9FFDDCFEAFF040EE9
:102B9000E926000EEA22EF8C020EE15C02E2E16A15
:102BA000E552E16EE552E7CFD9FF12006D980101C1
:102BB00014BF2BD019AF09D0020E106F2F5101E1B5
:102BC00058DF01012D6B2C6B1FD005C1E9FF06C139
:102BD000EAFFEE52080EEF6E05C1E9FF06C1EAFFFB
:102BE000020EE926000EEA22200EEE6E040EED6EB5
:102BF00005C1E9FF06C1EAFF8C0EEF6E0BC1E9FFCC
:102C00000CC1EAFF840EEF6E31D0040120AF0DD06D
:102C10000101010E106F2E5101E12BDF01012D6B1F
:102C20002C6B2B5101E1D4DE21D00101020E106F7B
:102C300005C1E9FF06C1EAFFEE52080EEF6E05C1BD
:102C4000E9FF06C1EAFF020EE926000EEA22200E85
:102C5000EE6E040EED6E05C1E9FF06C1EAFF840EBB
:102C6000EF6E2D6B2C6B2B5101E1B2DE1200D9CF30
:102C7000E6FFE1CFD9FFE652080EDF6E0101155DD8
:102C8000000E16590BE215C1DFFF0F5103E1010ED3
:102C90000F6F04D00F0502E1020E0F6FDF50146EAC
:102CA000156A1450155D156F15501659166F0BC126
:102CB000E9FF0CC1EAFFEE52DFCFEFFF280E1F6FD6
:102CC000040E206F14B11CD0DF5019E011C1F6FFC3
:102CD000112B12C1F7FF000E122313C1F8FF1323AB
:102CE0000800F550E66E1FC1E9FF20C1EAFF1F2B67
:102CF000000E2023E552E750EF6EDF06E5D717D030
:102D0000DF5015E011C1E9FF12C1EAFF112B000EDF
:102D10001223EF50E66E1FC1E9FF20C1EAFF1F2B0F
:102D2000000E2023E552E750EF6EDF06E9D7E552AB
:102D3000E552E7CFD9FF1200D9CFE6FFE1CFD9FFA7
:102D4000020EE12603C1E9FF04C1EAFFEE52EFCF14
:102D5000DFFFDFCF14F0145001011A5D000E1B5984
:102D600002E21AC1DFFFDF50146E156A14501A5DBB
:102D70001A6F15501B591B6F010EDB6ADF50F36E83
:102D8000010EDBCFF4FFF350F45C16E2010EDB50D2
:102D9000EA6A280FE96E040EEA22EF50E66E17C1C8
:102DA000E9FF18C1EAFF172B000E1823E552E75080
:102DB000EF6E010EDB2AE2D7000ED8801A55000E06
:102DC0001B5528E205C1E9FF06C1EAFFEE52080ED5
:102DD000EF6E05C1E9FF06C1EAFF020EE926000E0B
:102DE000EA22280EEE6E040EED6E03C1E9FF04C167
:102DF000EAFFEF50400B07E105C1E9FF06C1EAFF1A
:102E0000C80EEF6E06D005C1E9FF06C1EAFF880EC5
:102E1000EF6E2BD005C1E9FF06C1EAFFEE52080EA6
:102E2000EF6E05C1E9FF06C1EAFF020EE926000EBA
:102E3000EA22200EEE6E040EED6E05C1E9FF06C11A
:102E4000EAFF840EEF6E1C511D111E1109E007D020
:102E50001EC1FBFF1DC1FAFF01011C51F96EF8DF15
:102E60000101199F2B5101E1B3DD020EE15C02E289
:102E7000E16AE552E16EE552E7CFD9FF1200D9CF02
:102E8000E6FFE1CFD9FFE6520101148F010EE66E95
:102E9000E66AE66A710EE66E0F0EE66E05EC26F047
:102EA000146E050EE15E1450200EE66EE66AE66AC8
:102EB000000EE66E040EE66E05EC26F0146E050EAE
:102EC000E15E14506D8CDF6A020EDF5C10E2DF50B1
:102ED000EA6A260FE96E010EEA22EF6ADF50EA6A1B
:102EE000280FE96E010EEA22EF6ADF2AEDD7010E04
:102EF000E66EE66AE66A020EE66E010EE66E05EC26
:102F000026F0146E050EE15E14506D9C0101080E52
:102F10000B6F040E0C6F000E036F040E046F03C1E1
:102F200005F104C106F122C401F1015103E1100EC3
:102F3000006F13D0010EE66EE66A010EE66E010E1A
:102F4000E66E010EE66EE66A62EC24F0146E060E82
:102F5000E15E14500101200E006FE552E552E7CF0B
:102F6000D9FF1200800E0401205D01E0ACD0010108
:102F7000C00E146F04012351030A61E0010A10E03E
:102F8000030A03E00101146B9ED00101C60E116F0C
:102F9000490E126F000E136F120E156F166B93D041
:102FA000840E146E4A0E156E000E166E22C417F0B3
:102FB000186A196A030E0C6E0D6A0E6A17C007F0C4
:102FC00018C008F019C009F099EC25F004C017F0FA
:102FD00005C018F006C019F014501724F36E1550F0
:102FE0001820F46E16501920F86EF4CFF7FFF3CFC7
:102FF000F6FF0900F5CF11F10900F5CF12F1080035
:10300000F5CF13F111C1F6FF12C1F7FF13C1F8FF9D
:10301000020EF626000EF722F8220800F5CF15F171
:1030200011C1F6FF12C1F7FF13C1F8FF030EF62618
:10303000000EF722F8220800F5CF16F144D0040E56
:10304000225D3EE2870E146E4A0E156E000E166E5D
:1030500022C417F0186A196A030E0C6E0D6A0E6A04
:1030600017C007F018C008F019C009F099EC25F056
:1030700004C017F005C018F006C019F0145017244A
:10308000F36E15501820F46E16501920F86EF4CF18
:10309000F7FFF3CFF6FF0900F5CF11F10900F5CFE7
:1030A00012F10800F5CF13F111C1F6FF12C1F7FFBD
:1030B00013C1F8FF0800F5500101156F166B02D01F
:1030C0000101146B00D01200D9CFE6FFE1CFD9FF88
:1030D000020EE1260401286B296B20511F0B020A06
:1030E00012E0030A0DE0010A01E042D00101148F51
:1030F000040128810101210502E10401288338D05F
:103100000101148F35D00101148F040124BF10D0A8
:1031100024510F0BE96EEA6AD890E936EA36070EB9
:10312000E926010EEA22EECFDEFFEDCFDDFF0FD064
:1031300024510F0BE96EEA6AD890E936EA360B0E95
:10314000E926010EEA22EECFDEFFEDCFDDFFDECF76
:10315000E9FFDDCFEAFFEF50800B09E0DECFE9FFAA
:10316000DDCFEAFFEF50040B02E0010E286F00D024
:10317000010114AF07D0280E116F040E126F1481D5
:10318000020E156F020EE15C02E2E16AE552E16EA9
:10319000E552E7CFD9FF120070A015D003C1E9FFB7
:1031A00004C1EAFFEF5080080DE10BC1E9FF0CC13B
:1031B000EAFFEF50840806E103C1E9FF04C1EAFF1A
:1031C0008C0EEF6E7090689A1200698468986D8218
:1031D0000101010E226F000EE66EE66AE66EE66AF7
:1031E000750EE66EE66A62EC24F0146E060EE15E81
:1031F000145012000101226B000EE66EE66AE66EC4
:10320000E66A740EE66EE66A62EC24F0146E060E50
:10321000E15E14506D92699468A402D06894FCD762
:103220001200D9CFE6FFE1CFD9FFE65201012D0E02
:103230002A6FFD0E231553E17E0E2315E8407F0B08
:10324000040DF3CF03F1F4CF04F1000E0327040EB5
:10325000042303C105F104C106F1057503C1E9FFAB
:1032600004C1EAFFEF503C0BE842E8420D0835E1AB
:10327000DF6A080EDF5C23E203C1E9FF04C1EAFF55
:10328000020EE926000EEA22EE50EFCFEAFFE96EC9
:10329000EF50E66EDF50EA6A200FE96E040EEA2274
:1032A000E552E750EF6E03C1E9FF04C1EAFF020EE9
:1032B000E926000EEA22EE2AEF22DF2ADAD703C13E
:1032C000E9FF04C1EAFF020EE926000EEA22200E01
:1032D000EE6E040EED6E0DD801D03AD805D0FD0E7D
:1032E0002315040801E159D8E552E552E7CFD9FF8B
:1032F000120001010F6B2B6B2E6B2F6B256B106B6C
:103300000BC1E9FF0CC1EAFFEF9E0B750BC1E9FF92
:103310000CC1EAFFEF9E0B7505C1E9FF06C1EAFF8C
:10332000EF9E146B156B166B196B1A6B1B6B92D897
:10333000000EE66EE66AE66EE66A030EE66EE66A82
:1033400062EC24F0146E060EE15E1450D6EF15F018
:10335000020E0101105D02E1EFDC1ED0106B255161
:103360001AE105C1E9FF06C1EAFFEE52080EEF6E51
:1033700005C1E9FF06C1EAFF020EE926000EEA22B6
:10338000200EEE6E040EED6E05C1E9FF06C1EAFFE8
:103390008C0EEF6E01D0256B1200D9CFE6FFE1CF86
:1033A000D9FFE6520BC1E9FF0CC1EAFFEF50400B19
:1033B00001E0010EDF6E01010B75080E005D09E1F1
:1033C00022C46EFF6E5003E0100E006F02D0040E98
:1033D000006F100528E10BC1E9FF0CC1EAFF020EE6
:1033E000E926000EEA22280EEE6E040EED6E3FDC9A
:1033F000020E01010F5D07E10BC1E9FF0CC1EAFFFD
:10340000840EEF6E0FD0DF5007E10BC1E9FF0CC156
:10341000EAFFC80EEF6E06D00BC1E9FF0CC1EAFF50
:10342000880EEF6E12D019AF0FD01C511D111E1156
:1034300009E007D01EC1FBFF1DC1FAFF01011C51AD
:10344000F96EF8DF0101199F106BE552E552E7CFE5
:10345000D9FF120004012051600BE842E842E84223
:10346000E842E842000901E058D021510C0A54E03A
:103470000B0A43E00C0A35E0010A26E00B0A22E0C1
:10348000020A20E0030A1CE0080A10E0010A0CE02E
:103490000F0A08E0030A01E03FD00101148F080E73
:1034A000006F3BD05FDD39D0EADC37D00101010E7F
:1034B000116F010E126F1481010E156F148F2DD034
:1034C00003DE2BD02BD829D024510101116F126BB0
:1034D000020E1127010E12231481010E156F148F95
:1034E0001CD00101148F04012451EA6A020FE96E15
:1034F000010EEA2222C4EFFF10D0000EE66EE66A4B
:10350000E66EE66A020EE66EE66A62EC24F0146E7F
:10351000060EE15E145001D000D01200D9CFE6FFB4
:10352000E1CFD9FF050EE1260401220510E120516B
:103530001F0B00090CE10101148F030E0401215D32
:1035400004E10101010E216F02D00101216B040190
:10355000225101E020D120511F0B020801E01BD1B4
:1035600024510F0B000901E116D124510F0B010862
:1035700001E211D1200E0101005D01E00CD1148F98
:10358000040124BF1AD024510F0BE96EEA6AD890C7
:10359000E936EA36070EE926010EEA22EECFDEFF13
:1035A000EDCFDDFF24510F0BEA6A280FE96E010E03
:1035B000EA22020EEFCFDBFF19D024510F0BE96E88
:1035C000EA6AD890E936EA360B0EE926010EEA22BD
:1035D000EECFDEFFEDCFDDFF24510F0BEA6A260FA1
:1035E000E96E010EEA22020EEFCFDBFFD950020F87
:1035F000E96EDACFEAFFEF50010B03E1000EDF9432
:1036000001D0DF8424BF10D024510F0BE96EEA6A89
:10361000D890E936EA36070EE926010EEA22DECF17
:10362000EEFFDDCFEDFF0FD024510F0BE96EEA6AFC
:10363000D890E936EA360B0EE926010EEA22DECFF3
:10364000EEFFDDCFEDFF030E215D23E1DECFE9FFCD
:10365000DDCFEAFFEF50800B13E024BF09D02451E7
:103660000F0BEA6A280FE96E010EEA22EF8208D0FA
:1036700024510F0BEA6A260FE96E010EEA22EF824F
:10368000840E146EDECFE9FFDDCFEAFF1450EF1297
:1036900082D0DF74DECFE9FFDDCFEAFFEF50800B91
:1036A0001BE0DECFE9FFDDCFEAFFEF9EDECFE9FFD3
:1036B000DDCFEAFFEF8C020EE66EE66ADECFE6FFB4
:1036C000DDCFE6FF050EE66EE66A62EC24F0146ECE
:1036D000060EE15E145005D0DECFE9FFDDCFEAFF34
:1036E000EF8CDF74D950020FE96EDACFEAFFEF50AA
:1036F000020B07E1DECFE9FFDDCFEAFFEF50800BE1
:103700002DE0040124BF09D024510F0BEA6A280FD1
:10371000E96E010EEA22EF9208D024510F0BEA6AFB
:10372000260FE96E010EEA22EF923B0E146EDECFF9
:10373000E9FFDDCFEAFF1450EF16020EE66EE66AEF
:10374000DECFE6FFDDCFE6FF050EE66EE66A62EC51
:1037500024F0146E060EE15E145008D03B0E146E79
:10376000DECFE9FFDDCFEAFF1450EF16040124514C
:103770000F0B156A700F146E0F0E1522030E14C076
:10378000DBFF040E15C0DBFF030EDBCFE9FF040EE9
:10379000DBCFEAFFEF90050EE15C02E2E16AE55261
:0A37A000E16EE552E7CFD9FF1200F9
:0637AA00400EE66E300E39
:1037B000E66E040EE66EE66A010EE66E80EC13F02D
:1037C000146E050EE15E1450F3CF99F0F4CF9AF029
:1037D0000DC19BF00EC19CF00001606B6169626BD2
:1037E000636BA26BAA6BAB6BAC6BAD6BAE6BAF6B71
:1037F000B06BB16B010EA36F9F6BA06B726B010E70
:10380000725D22E27251EA6AA10FE96E000EEA22AD
:10381000EF6A16EC04F0000912E0EAEC0DF0F3CFC9
:1038200014F0F4CF15F01450151009E00001725196
:10383000AFEC26F0F35000019F13F450A01349ECB5
:1038400022F00001722BDBD71200040120511F0B64
:10385000010801E054D0245101E051D02151FE0A69
:1038600038E0010A01E04BD02251231103E1265137
:10387000271101E044D00001606B6169626B636BEA
:10388000010EA36F010109510A1102E1000E08D0D7
:1038900009C1E9FF0AC1EAFFEF50800B01E0010E08
:1038A000000913E1400EE66E300EE66E040EE66E81
:1038B000E66A010EE66E80EC13F0146E050EE15E12
:1038C0001450F3CF99F0F4CF9AF00101800E146FE9
:1038D00016D02251231105E1010E261901E12751CD
:1038E00001E00DD00401286B0101280E116F040EB8
:1038F000126F010E156F166BC10E146F00D01200FF
:10390000D9CFE6FFE1CFD9FFE652200E0101005DDD
:1039100002E0000E21D1A09A00016051030A01E1EA
:10392000C2D0010A01E1AED0030A01E1A4D0010A2C
:1039300001E003D199519A1102E1000E08D099C01B
:10394000E9FF9AC0EAFFEF50800B01E0010E000989
:1039500001E090D0DF6A1F0EDF5C13E2DF50EA6AFD
:10396000300FE96E040EEA22EF50E66EDF50EA6A8D
:10397000650FE96E000EEA22E552E750EF6EDF2A8E
:10398000EAD799C0E9FF9AC0EAFFEE52EF501F084C
:1039900061E1550E0001651908E1530E661905E154
:1039A000420E671902E1430E681954E1010EA36F3C
:1039B0007251000840E3735110083DE3010E735D3E
:1039C0003AE33F0E711537E10401550E4F6F530E68
:1039D000506F420E516F530E526F69C053F46AC05C
:1039E00054F46BC055F46CC056F4576B586B596B5C
:1039F0005A6B5B6B00016169626B636B646B030EF6
:103A0000745D06E08791879387958797916B926B9A
:103A100071AF03D0010E606F02D0020E606F6D5166
:103A20006E116F11701102E0A26B02D0010EA26F35
:103A300074C061F00ED0010EE66EE66E03EC14F079
:103A4000E552E552E66A010EE66E03EC14F0E5522B
:103A5000E55210D0010EE66EE66E03EC14F0E5526E
:103A6000E552E66A010EE66E03EC14F0E552E5520B
:103A70000001A36B6DD075D8FF0803E10001030EB0
:103A8000606F66D06ED8FF080DE104015B5107E15D
:103A90005751581159115A1102E0020E5B6F000183
:103AA000030E606F55D001010D510E1102E1000EA1
:103AB00008D00DC1E9FF0EC1EAFFEF50800B01E015
:103AC000010E000901E044D00D0EE66E4F0EE66EC9
:103AD000040EE66E010EE66EE66E80EC13F0146ED8
:103AE000050EE15E1450F3CF9BF0F4CF9CF0000183
:103AF00099519A1102E1000E08D099C0E9FF9AC0CD
:103B0000EAFFEF50800B01E0010E000913E1400EC7
:103B1000E66E300EE66E040EE66EE66A010EE66EA6
:103B200080EC13F0146E050EE15E1450F3CF99F0A3
:103B3000F4CF9AF00001606B0BD0606B0401020EB1
:103B40005B6FE66A010EE66E03EC14F0E552E55297
:103B5000A08A0001605100D0E552E552E7CFD9FFBD
:103B6000120016EC04F0000909E000017251EA6A43
:103B7000A10FE96E000EEA22EF0411E1000172517B
:103B8000AFEC26F0F3CF14F0F4CF15F0141E151E91
:103B9000145000019F171550A01733D82ED0725122
:103BA000AFEC26F000019F51F314146EA051F414F1
:103BB000156E1450151020E1EAEC0DF0F3CF14F05F
:103BC000F4CF15F01450151015E000017251AFEC50
:103BD00026F0F35000019F13F450A01387918783C0
:103BE00087858797280E916F926B0401010E5B6F9A
:103BF00031D801D006D801D02DD80001615100D0B4
:103C0000120000016151FD0A22E0EF0A1EE00C0AD9
:103C100016E01E0A14E0030A06E07F0EE66E12ECC0
:103C200023F0E55216D049EC22F0000187918783FA
:103C3000879587973A0E916F926B0CD80AD0040142
:103C4000010E5B6F0001616904D004D802D002D874
:103C500000D01200D9CFE6FFE1CFD9FF0A0EE1264E
:103C600000016151FE0A01E194D1030A01E125D16D
:103C7000D20A01E11AD1340A01E117D11B0A01E18C
:103C8000F4D01E0A01E1E0D0040A01E1C2D0190A11
:103C900001E193D0260A4EE0370A11E0380A09E024
:103CA000020A01E076D1D0D9000902E10001616980
:103CB00075D1B8DA000902E1000161696FD1A2058E
:103CC00002E161696BD177C0A5F078C0A4F0A4C00F
:103CD00014F0A5C015F0166A176A14C0E6FF15C0E7
:103CE000E6FF16C0E6FF17C0E6FFF5DBE552E5523A
:103CF000E552E552000901E051D1240EE66EE66A74
:103D000057D9E552E552240EE66EE66AFE0EE66EDF
:103D10004C0EE66E000EE66E000EE66E060EE66EC9
:103D2000E2EC25F0146E070EE15E14500001FD0E6A
:103D3000616F34D123EC04F0060E06C0DBFF070EE2
:103D400007C0DBFF080E08C0DBFF090E09C0DBFF60
:103D50001DEC04F0F3CF14F0F4CF15F0020E14C0F4
:103D6000DBFF030E15C0DBFF040EDB6A050EDB6A0A
:103D7000090EDBCF00F6080EDBCF01F6070EDBCF16
:103D800002F6060EDBCF03F6050EDBCF04F6040EBB
:103D9000DBCF05F6030EDBCF06F6020EDBCF07F610
:103DA000080E0001A46FA56BE66EE66A01D9E55224
:103DB000E5520001FD0E616FF1D0A20502E16169DB
:103DC000EDD0120EA46FA56BE66EE66AF1D8E5524F
:103DD000E552DF6ADF50146E156A120E145C000E95
:103DE000155813E2DF50EA6A850FE96E000EEA22E9
:103DF000EF50E66EDF50EA6A000FE96E060EEA2227
:103E0000E552E750EF6EDF2AE5D70001FD0E616F46
:103E1000C5D00601030E006F016BDAEC0CF000094F
:103E200002E0800E01D0000E0601026F036B040E4B
:103E30000001A46FA56BE66EE66ABAD8E552E552BA
:103E40000001FD0E616FAAD08781879387858797D0
:103E5000200E916F926B0401010E5B6F576B586BD4
:103E6000596B5A6B0001616999D0E66AE66AE66AA5
:103E7000E66A31DBE552E552E552E552000901E020
:103E80008DD0000187510F0B060806E104015B0588
:103E900003E10001616908D0FCDA0401576B586B3B
:103EA000596B5A6B0001616979D00401576B586BEB
:103EB000596B5A6B0001616971D09B519C1102E1F1
:103EC000000E08D09BC0E9FF9CC0EAFFEF50800BBA
:103ED00001E0010E00095CE1400E6D5D000E6E59BF
:103EE000000E6F59000E705909E3DE52400EDD6E70
:103EF0006D5F000E6E5B6F5B705B07D0010E6DC077
:103F0000DBFF6D6B6E6B6F6B706B010EDB50146EB5
:103F1000156A1450A45D1550A55909E3010EDB5034
:103F2000146E156A1450A45F1550A55B15D0DF6A96
:103F3000010EDB50DF5C10E2A451A51104E0A407E0
:103F4000000EA55B07D0DF50EA6A000FE96E060E8F
:103F5000EA22EF6ADF2AECD7010EDBCFE6FF000E84
:103F6000E66E060EE66E010EE66EE66E80EC13F06F
:103F7000146E050EE15E1450F3CF9BF0F4CF9CF06D
:103F800000016D516E116F11701102E1616906D06F
:103F900005D07F0EE66E46DBE55200D00A0EE15CEE
:103FA00002E2E16AE552E16EE552E7CFD9FF120085
:103FB000D9CFE6FFE1CFD9FFFD0EDBCF14F0FE0E27
:103FC000DBCF15F0166A176A145000016D5D1550AD
:103FD0006E5916506F59175070590AE20401576B09
:103FE000586B596B5A6B6DC0A4F06EC0A5F028D009
:103FF000FD0EDBCF14F0FE0EDBCF15F0A451145CE8
:10400000A551155806E2FD0EDBCFA4F0FE0EDBCF66
:10401000A5F0A4C014F0A5C015F0166A176A6D0EBD
:10402000E96E000EEA6E1450EE5C0401576F1550F5
:10403000EE58586F1650EE58596F1750EE585A6F89
:10404000E552E7CFD9FF120000016251040A01E1F5
:10405000A0D0070A01E190D0010A3CE0030A30E059
:10406000010A01E0CFD076C0A9F077C0A8F078C0EF
:10407000A7F079C0A6F07BC0A5F07CC0A4F0A4C0D6
:1040800014F0A5C015F0166A176A090ED8901436F8
:10409000153616361736E806F9E114C0E6FF15C0E6
:1040A000E6FF16C0E6FF17C0E6FF15DAE552E55257
:1040B000E552E552000901E0B1D00001010E626F46
:1040C000A451A51102E1626BA9D0A407000EA55B63
:1040D000020E626F9B519C1102E1000E08D09BC042
:1040E000E9FF9CC0EAFFEF50800B01E0010E0009E0
:1040F00001E094D0000EE66E060EE66EA6C0E6FF66
:10410000A7C0E6FFA8C0E6FFA9C0E6FFB5EC07F030
:10411000146E060EE15E145001081BE0640E0001EF
:10412000645D03E2642B7AD014D00401020E5B6F4D
:1041300000018781878387958797916B926B010E2A
:10414000E66EE66E03EC14F0E552E5520001626B98
:1041500065D00001A62B000EA723A823A9230401E4
:10416000576B020E586F596B5A6B0001000E976F18
:10417000060E986F030E626F0401575158115911C2
:104180005A1104E10001010E626F48D00001040ED3
:10419000626F9B519C1102E1000E08D09BC0E9FFA9
:1041A0009CC0EAFFEF50800B01E0010E000901E026
:1041B00035D0400EE66E97C0E6FF98C0E6FF010ED0
:1041C000E66EE66E80EC13F0146E050EE15E1450A0
:1041D000F3CF9BF0F4CF9CF00001030E626F400E12
:1041E0006D5F000E6E5B6F5B705B400E0401575F8E
:1041F000000E585B595B5A5B400E00019727000E7A
:1042000098230CD00401020E5B6F010EE66EE66E81
:1042100003EC14F0E552E5520001626B00016251BB
:1042200000D0120000016351020A01E1E5D0060A44
:1042300001E1A5D0070A5DE0020A4AE0010A01E0B7
:1042400018D176C0A9F077C0A8F078C0A7F079C0DF
:10425000A6F07BC0A5F07CC0A4F0A4C014F0A5C05B
:1042600015F0166A176A090ED890143615361636E8
:104270001736E806F9E114C0E6FF15C0E6FF16C0E0
:10428000E6FF17C0E6FF27D9E552E552E552E552B1
:10429000000901E0FAD0DAEC0CF0000916E00401A4
:1042A000010E5B6F00018781878387858797270EC3
:1042B000916F926BE66A010EE66E03EC14F0E55224
:1042C000E5520001636B6351E3D00001010E606FA2
:1042D000A451A51102E1636BD8D0030E636F000EE9
:1042E000976F060E986F0401576B020E586F596B4B
:1042F0005A6BD880000E04015755000E5855000E19
:104300005955000E5A5528E2000199519A1102E1BF
:10431000000E08D099C0E9FF9AC0EAFFEF50800B69
:1043200001E0010E000901E0B0D0400EE66E97C03A
:10433000E6FF98C0E6FFE66A010EE66E80EC13F039
:10434000146E050EE15E1450F3CF99F0F4CF9AF09D
:104350000001040E636F13D0DAEC0CF000090BE0DF
:104360000401010E5B6F0001879187838795879712
:10437000270E916F926B0001020E636F86D09951E8
:104380009A1102E1000E08D099C0E9FF9AC0EAFF35
:10439000EF50800B01E0010E000901E076D099C0DA
:1043A000E9FF9AC0EAFFEE52EFCF14F0156A166AE1
:1043B000176A14506D5F15506E5B16506F5B175087
:1043C000705B99C0E9FF9AC0EAFFEE52EFCF14F09C
:1043D000156A166A176A14500401575F1550585B26
:1043E0001650595B17505A5B400E00019727000E7C
:1043F0009823030E636F49D004015B512FE1000144
:10440000A651A711A811A91102E1010E01D0000EB9
:10441000E66E000EE66E060EE66EA6C0E6FFA7C0CC
:10442000E6FFA8C0E6FFA9C0E6FF89EC0CF0146E19
:10443000070EE15E1450010811E0640E0001645D96
:1044400003E2642B22D00AD00401010E5B6F00014D
:104450008781878387958797916B926B0001A62B45
:10446000000EA723A823A923A407A55B010E636F51
:104470000CD00401020E5B6FE66A010EE66E03ECDF
:1044800014F0E552E5520001636B0001635100D066
:104490001200000185918593859585978589858B87
:1044A000858D859F866B8791879387958797879B57
:1044B000879D879F886B896B8A6B8B6B0A0E8C6FCD
:1044C0008D6B8E6B8F6B906B916B926B936B946B10
:1044D000956B966B1200D9CFE6FFE1CFD9FF030EA3
:1044E000E126FB0EDBCF14F0FC0EDBCF15F0FD0E4A
:1044F000DBCF16F0FE0EDBCF17F0145015101610A0
:10450000171006E1010EF36E020EF3CFDBFF02D0AF
:10451000020EDB6A0001A20505E1020EDB0402E1E6
:10452000000E74D0D950FB0FE96EFF0EDA20EA6E50
:104530006D51EE1809E16E51EE1806E16F51EE185B
:1045400003E17051EE1800E10DE1600506E12A0E6D
:10455000615D02E0000E5AD005D02A0E615D02E1D5
:10456000000E54D0D950FB0FE96EFF0EDA20EA6E30
:104570006D51EE5C6E51EE586F51EE587051EE5821
:1045800004E2DE52010EDD6E02D0010EDB6A020E85
:10459000605D1DE12A0E615D06E0020EDB5003E165
:1045A000050EDF6E13D0A20503E1010EDF6E0ED003
:1045B000020EDB0403E1040EDF6E08D0010EDB0403
:1045C00003E1040EDF6E02D0050EDF6E19D02A0E55
:1045D000615D03E1030EDF6E13D0A20503E1010E5E
:1045E000DF6E0ED0020EDB0403E1020EDF6E08D098
:1045F000010EDB0403E1020EDF6E02D0030EDF6E5C
:10460000DFCFE6FF0FD8E552DF5000D0146E030E67
:10461000E15C02E2E16AE552E16E1450E552E7CF57
:10462000D9FF1200D9CFE6FFE1CFD9FFE652000152
:104630009B519C1102E1000E08D09BC0E9FF9CC079
:10464000EAFFEF50800B01E0010E00090FE19951E4
:104650009A1102E1000E08D099C0E9FF9AC0EAFF62
:10466000EF50800B01E0010E000901E06DD060C049
:10467000DFFF6169626B636B6DC057F46EC058F405
:104680006FC059F470C05AF40401010E5B6F000151
:10469000030E606FFE0EDB507F0A35E07A0A28E0D9
:1046A000010A1EE0070A11E0010A07E0030A01E01F
:1046B0004BD00401020E5B6F47D0010EE66EE66E32
:1046C00003EC14F0E552E5523FD00401020E5B6F9B
:1046D000010EE66EE66E03EC14F0E552E55234D0BE
:1046E000E66A010EE66E03EC14F0E552E5522CD0BA
:1046F0000401020E5B6FE66A010EE66E03EC14F035
:10470000E552E55221D0C5DE000187818793878578
:104710008797200E916F926B020EDF5C0DE16D5159
:104720006E116F11701108E0E66A010EE66E03EC7F
:1047300014F0E552E55207D0010EE66EE66E03EC8A
:1047400014F0E552E55200D0E552E552E7CFD9FF2B
:02475000120055
:0E475200DACFE4FFE2CFDAFFE9CFE4FFEACFEF
:10476000E4FFF6CFE4FFF7CFE4FFF8CFE4FFF5CFA7
:10477000E4FFF3CFE4FFF4CFE4FFFACFE4FFFBCF95
:10478000E4FF00EE00F0140EE80403E3EECFE4FFD4
:10479000FBD700EE14F0100EE80403E3EECFE4FFC5
:1047A000FBD7E65291EC12F0E55200EE23F0100E2A
:1047B000E80403E3E5CFEDFFFBD700EE13F0140EA2
:1047C000E80403E3E5CFEDFFFBD7E5CFFBFFE5CF43
:1047D000FAFFE5CFF4FFE5CFF3FFE5CFF5FFE5CF37
:1047E000F8FFE5CFF7FFE5CFF6FFE5CFEAFFE5CF2E
:1047F000E9FFE5CFDAFF1100D8CFE4FFE0CFE4FF17
:10480000E46EDACFE4FFE2CFDAFFE652E552E5CF1D
:10481000DAFFE550E5CFE0FFE5CFD8FF100005D87F
:10482000D1EC14F008D8FED712000F0EC1122DECF7
:1048300004F005EF12F0200E0101E76E0019E8AE5A
:1048400002D0E73402D0E750005D03E36D50020B65
:1048500001E002D080EC1CF01200120012001200E5
:10486000120025EF1CF012001E0EE66E010EE66E21
:1048700049EC13F0E552E552D5EF1BF0010121059B
:1048800020E1010122051DE1A09AE8DF6D920101FE
:10489000226B0001100EFA6F0E0EFB6FFA07000E6E
:1048A000FB5BFA51FB11FAE16D84080EFA6F070EFB
:1048B000FB6FFA07000EFB5BFA51FB11FAE16D94F6
:1048C000A08A1200D9CFE6FFE1CFD9FFFD0EDBCFE2
:1048D00008F0FE0EDBCF09F0050E081801E10950C3
:1048E00039E0E868081802E17F0E091831E0030E8C
:1048F000081801E109502AE0020E081801E10950E8
:1049000023E0010E081801E109501CE0740E08189C
:1049100001E1095015E0750E081801E109500EE09B
:10492000730E081801E1095007E0720E081801E142
:10493000095001E042D041D092DF3FD08EDF3DD020
:104940008DDF3BD091DF39D08EDF37D08ADF35D095
:1049500087DF33D00001A3510FE1010EE66EE66E52
:1049600003EC14F0E552E552E66A010EE66E03EC44
:1049700014F0E552E55220D0FB0EDBCF14F0FC0E14
:10498000DBCF15F001010951141802E10A51151885
:1049900013E1400EE66E300EE66E040EE66EE66A39
:1049A000010EE66E80EC13F0146E050EE15E1450FD
:1049B000F3CF99F0F4CF9AF000D0010E00D0E55279
:0649C000E7CFD9FF120051
:0A49C6001201000200000008D804EE
:1049D000090001000102030109022000010100C0D9
:1049E0003209040000020806500007058102400059
:1049F00001070501024000010403090434034D00CE
:104A00006900630072006F00630068006900700055
:104A1000200054006500630068006E006F006C00A9
:104A20006F0067007900200049006E0063002E00CF
:104A30003A034D006900630072006F006300680074
:104A40006900700020004D006100730073002000B9
:104A5000530074006F007200610067006500200061
:104A6000440072006900760065001A0331003200CC
:104A7000330034003500360037003800390030008C
:104A800039003900D84900F84900FC4900304A0093
:034A90006A4A006F
:0C4A94002A0EF66E080EF76E000EF86E8B
:104AA00000010900F550F56F0900F550F66F03E1BC
:104AB000F56701D03DD00900F550F06F0900F550C1
:104AC000F16F0900F550F26F09000900F550E96E29
:104AD0000900F550EA6E090009000900F550F36F6E
:104AE0000900F550F46F09000900F6CFF7F0F7CF91
:104AF000F8F0F8CFF9F0F0C0F6FFF1C0F7FFF2C020
:104B0000F8FF0001F35302E1F45307E00900F55008
:104B1000EE6EF307F8E2F407F9D7F7C0F6FFF8C036
:104B2000F7FFF9C0F8FF0001F507000EF65BBFD7ED
:024B3000120071
:0E4B320009C013F008C012F007C011F00750C0
:104B40000C02F4CF05F0F3CF04F008500D02F4CFBF
:104B500007F0F3CF06F00C02F3500526F4500622BE
:104B6000E86A072211500D02F3500526F450062280
:104B7000E86A072209500C02F3500626F450072277
:104B800009500D02086AE86A0822F3500726F4501B
:104B9000082211500E02F3500626F4500722096A2B
:104BA000E86A0822092212500E02F3500726F45038
:104BB0000822E86A092213500E02F3500826F45026
:044BC0000922000CBA
:0C4BC400FB0EE3CFF6FFFC0EE3CFF7FF83
:104BD000FD0EE3CFF8FFFE0EE3CFE9FFFF0EE3CFBC
:104BE000EAFFE9CFF3FFEACFF4FFF90EE35003E168
:104BF000FA0EE35009E0F90EE30602E2FA0EE306CC
:104C00000900F5CFEEFFF1D71200FE0EE3CFE9FF6A
:104C1000FF0EE3CFEAFFE9CFF3FFEACFF4FFFB0E8D
:104C2000E35003E1FC0EE35009E0FB0EE30602E271
:0E4C3000FC0EE306FD0EE350EE6EF1D712000F
:024C3E0006501E
:104C40000B02F3CF02F0F4CF03F00C02F350032673
:104C5000000EF420046E06500D02F3500426000EE0
:104C6000F420056E06500E02F350052607500B0285
:104C7000F3500326F4500422000E052207500C02C4
:104C8000F3500426F450052207500D02F350052678
:104C900008500B02F3500426F450052208500C0271
:0E4CA000F350052609500B02F35005261200B2
:024CAE0000956F
:104CB000000001F900000887040009AF00010A1B89
:104CC00000010CC301000DAF020010FF000011FF36
:104CD000000112FF000118FF000119FF000120FF71
:104CE000000021FF000026DF0100377300003A2595
:0E4CF00004003B25000029FF040017FF000010
:024CFE00008034
:104D00000402200000004D6963726F6368704D619A
:104D100073732053746F72616765202020203030D8
:024D2000303130
:0E4D2200000EF36E00EE00F0080E01D8120035
:104D3000EA6002D0EE6AFCD7F350E9601200EE6A36
:024D4000FCD79E
:0E4D420013EE00F023EE00F0F86A019C4AEC3C
:0E4D500025F0BAEC26F00FEC24F0FBD7120091
:024D5E00F36AF6
:104D6000F46AF32A0F0B05E0D890F336F436E80422
:044D7000FBE1120051
:024D740012002B
:020000040030CA
:0100000024DB
:010001000EF0
:010002003FBE
:010003001EDE
:010005008179
:010006008178
:010008000FE8
:01000900C036
:01000A000FE6
:01000B00A054
:01000C000FE4
:01000D0040B2
:00000001FF
